:03000000021D528C
:0C1D520078FFE4F6D8FD7581E20200364F
:01001A0022C3
:061A4B008B2C8A2D892E70
:101A5100751A027F48121BC7121D97EF20E0F9ABE0
:101A61002CAA2DA92E1207BC7874E6FE08E6FDED1E
:011A7100FF75
:011A72002251
:100FC500434647002D53322D0052415445434C5260
:100FD50020554E49544C495445545249475452455D
:100FE500565354525453544F505A45524F424155FB
:100FF5004444464C54534156455253542050432083
:10100500205F3120735F3220735F35207331207389
:101015002032207320352073203130207333302067
:101025007331206D2032206D2035206D2031302028
:101035006D3330206D312068200000000100020072
:1010450005000A001400320064012C025804B00B9C
:10105500B8177046508CA00102040810304665652B
:1010650074596172644D6574724F6666204F6E20C7
:10107500204E6F2020596573204F66662054696D98
:1010850065416C7420547269674F666620547269B5
:0910950067537472745265632004
:101B0A0025E0243EF582E43410F58322052EE52EE5
:101B1A00C3940222A62EE52E75F004A42208F60824
:041B2A00F608F622A1
:10177100789476AB0876CD08760008760AE408F608
:1017810008760108F6087664087640121B2708F6E9
:1017910078A2F608760A08F608763C08F608761468
:0F17A10008F608760F121B2778AF7605021AE6B6
:10197000751E1D751FC01216297895E664CD70047A
:1019800018E664AB600312177178AEE6FFF46003EB
:0F199000EF700478AE760178AFE6B4FF0276050B
:01199F002225
:0D1D2800C2AF7DC07C1DE4FF121C6DD2AF68
:011D3500228B
:101629007539FF851E3A851F3B753C00753D007570
:101639003E94E4FFAB39AA3AA93B8F827583001225
:10164900078FAB3CAA3DA93E8F827583001207CE56
:101659000FBF1CE078ADE6FFF46003EF700478ADCE
:02166900760108
:01166B00225C
:101AE6007D01E4FF121B6F121D28C2AF7F947B1C81
:101AF6007DC07C1D121C77D2AF7F0212189EE4FDBA
:041B0600FF021B6F50
:10051C00E4F52C7BFF7A0F79C51217317F05121881
:10052C009EA297829650FAA2969217A2979218E5DD
:10053C002C75F004A424CEF9740F35F0FA7BFF125D
:10054C0017317F0512189E852C2DE4F52E7BFF7A32
:10055C000F79C9121731E52CB40A0040030205EAE1
:10056C00900573F82828730205910205EA0205B27A
:10057C000205BA0205BE0205C60205CE0205D2026C
:10058C0005DA0205E27F01EF121B0A7896E6FC08F9
:10059C00E6FD7401936D7003E4936C70028F2E0F63
:1005AC00BF0FE40206707898E6F52E020693789950
:1005BC00800278A1E6F52E0206AD78A0E6F52E02B3
:1005CC0006DB78AA800278ABE6F52E0206F878AC4A
:1005DC00E6F52E02072D78AFE6F52E020753E52C33
:1005EC00652D600302053BA217309601B35013A290
:1005FC0096921730960C052CE52CC3940D4003E411
:10060C00F52CA218309701B350D4A29792183097BA
:10061C00CDE52CB40D0050C690062BF8282873029B
:10062C00065202067B02068102069F0206B90206EA
:10063C00CD0206E602070302071B0207410207640C
:10064C0002076A020770052EE52EC3940F4003754E
:10065C002E01E52E121B0AE493FF7401937896CFBA
:10066C00F608EFF6121B202402F97410020736125A
:10067C0014550205EA052EE52EC394034003E4F558
:10068C002E7898A62EE52E75F004A42462F9741029
:10069C00020736121B164003E4F52E7899A62EE5B8
:1006AC002E75F004A4246EF97410020736121B1672
:1006BC004003E4F52E78A1121B1E246EF9741080F1
:1006CC0069121B164003E4F52E78A0A62EE52E75B4
:1006DC00F004A42476F974108050052EE52EC394F2
:1006EC00044003E4F52E78AAA62EE52E75F004A49A
:1006FC00247EF974108033052EE52EC39403400339
:10070C00E4F52E78AB121B1E247EF97410801B05A9
:10071C002EE52EC394044003E4F52E78ACA62EE50A
:10072C002E75F004A4248EF9741035F0FA7BFF12A8
:10073C0017310205EA052EE52EC394064003E4F5B5
:10074C002E78AFA62EE52E90105C9375F018A4FFB2
:10075C00AEF01212830205EA1217710205EA121AA0
:0A076C00E60205EA43A2080205EACE
:0A1D6A004552415300444F4E45001E
:101CF7007896E6F55008E6F55122E565AE64780674
:011D070022B9
:1011F700C215C21678AEE6FFE4FCFDFEFB7A20F9C5
:10120700F81207F08F6B8E6A8D698C68E47B40FA61
:10121700F9F812087B8E628F63E4F52DF52EC3E58E
:101227002E9563E52D9562501CE52C64816016AF01
:101237002EAE2D1219A0121C598F2C052EE52E70DB
:10124700DD052D80D9E52CB48108E52E152E700219
:10125700152DE52E65637004E52D6562700CD215BA
:10126700121D36E4F564F5658007852D64852E65C6
:0B127700E4F566F567754F80121CF768
:011282002249
:1019A000C3EF9563EE95625024EF7806C333CE33D0
:1019B000CED8F9FD751A02EE7874F6CFEDCFEF08A8
:0D19C000F67F50121C17121D97EF20E0F962
:0119CD0022F7
:031BFD00CDEFCD5C
:101C0000751A02EE7874F6ED08F67F50121C171262
:061C10001D97EF20E0F932
:011C160022AB
:101C5900751A017F50121BC7121D97EF20E0F97802
:031C690074E6FF1F
:011C6C002255
:101C4400121BFDE4FFFE0FBF00010EBE0FF8BFA084
:041C5400F5121C5910
:011C58002269
:0618D400CBEFCBCAEECA07
:1018DA00301503301627751A03EA7874F6EB08F602
:1018EA0008EDF67F50121C17121D97EF20E0F9E45D
:0D18FA00FFFE0FBF00010EBE0FF8BFA0F5EE
:0119070022BD
:1016AF00752F0075300075314FE4F52E121D01C3F3
:1016BF0033CE33CED8F97C00252EFFEC3EFEAB2F78
:1016CF00AA30A931852E8275830012078FFD12185B
:1016DF00D4052EE52EC3940640D2756600756706B5
:0116EF0022D8
:101384008E2C8F2D121D01C333CE33CED8F9256791
:10139400FFE5663EFEEEC0E0EFC0E0E52CFDD0E0E8
:1013A400FFD0E0FE1218D40567E5677002056612E7
:1013B4001D01C333CE33CED8F92567FFE5663EFE63
:1013C400AD2D1218D40567E567700205660553E56F
:1013D4005370020552C3E5679440E56694004017D4
:1013E400E4F566F5670565E565700205649563E5F2
:0813F4006495624002D215224B
:10145500E4F566F5677BFF7A1D796A121731D216B6
:10146500E4F539F53AC3E53A9563E53995625021D6
:10147500E53AAE397806C333CE33CED8F9F5678E63
:10148500667D81FF1218D4053AE53A70D805398092
:10149500D4C2167BFF7A1D796F121731E4F564F516
:0714A50065F566F567C2154D
:0114AC00221D
:1013FC00E4F539F53AF53BF53CC3E53C9563E53B43
:10140C0095625044E53A6481603EAF3CAE3B1219A4
:10141C00A0121C598F3AE53A64807022AF39053915
:10142C00FCFDFEFBFAF9120D9C7F2C12001EAE3B4C
:10143C00AF3CE4FCFDFBFAF9120D9C121D87053C38
:08144C00E53C70B5053B80B1E1
:011454002275
:02159E008F3983
:1015A000E4F53AF53BF53CF53DC3E53D9563E53C97
:1015B00095625030E53B6481602AAF3DAE3C121924
:1015C000A0121C598F3BE53BB4800FE53A6539709A
:1015D00007AF3DAE3C0219A0053A053DE53D70C997
:0415E000053C80C581
:0115E40022E4
:1016F000121CF778A1E6F554E4F552F5531216AF33
:1017000085646C85656D7F01121A9A30021A78A47F
:10171000E6FE08E6FFE4FCFD7B64FAF9F81207F048
:101720008F618E608D5F8C5E300505C205121C2EA8
:011730002296
:10182A0085642C85652DE56745666008052DE52DDF
:10183A007002052C856C64856D651216AF852C6463
:10184A00852D65C3E52D9563E52C95624007E4F582
:0A185A0064F565D2157F02021A9AA8
:101C6D00740478FF769612FF0322740078FF76963F
:041C7D0012FF03222D
:0300330002109E1A
:0D109E00C0E0C0F0C083C082C0D075D00893
:1010AB00E5D954F8FF12099410D80810D81010E79E
:1010BB001811022010E928110230110438110A40CE
:1010CB001102481123501140580000114E851DDAB2
:1010DB00C2DDC2DC751B00751C008070800EE51A2A
:1010EB0070028056051CE51C7002051B1200268F32
:1010FB00DAC2DDC2DC80558016D2DDC2DC804DC287
:10110B00DDC2DCE51A7004C2DA8041D2DA803DC25E
:10111B00DDD2DC7518048034AFDA121D5E051CE5D8
:10112B001C7002051BC2DDC2DCE51A7004C2DA803A
:10113B001BD2DA8017AFDA121D5EC2DDD2DC751856
:0E114B00028009751804C2DDC2DCD2DAC2DBF4
:0B115900D0D0D082D083D0F0D0E032A4
:1019F90043910C43920CE4F5DBEF25E0F5DB30175E
:101A09000343DB0175DD1775DC1775D84453F8FE00
:091A190053F7FEE4F518D2E822AF
:101C1700E51830E002FF22E4F519751803EF25E017
:071C2700F51DD2DD7F022252
:101BC700E51830E002FF22E4F519151A751805EF3C
:0B1BD70025E04401F51DD2DD7F022255
:061D970020DBFDAF182265
:0D002600151AAF19051974742FF8E6FF22A2
:0C1D5E0074742519F8EFF60519151A2207
:101D0800E4F5847585FF53913FF592F5A475A5FF19
:011D180022A8
:1019CE00811902006F035D5733767E437F771004D3
:1019DE00007B3E6C1F7C78773B020F382C5A1A6FB7
:0B19EE00797518763C0E2F4E2B375DEC
:101864004EFECCEFCC0F74742CF8EEF6EDC433229C
:101874009019DEE493FF78DAF608EFF608F608F636
:1018840022E493FF74DA2EF8EFF60E22EE3395E09D
:0A189400FDFC227B007A0079D522CA
:10116400E4FF0F2474F876CD0F74742401F87680AC
:101174000F74742402F876E00F74742403F876F87C
:1011840030190A0F74742404F87671800ACEEFCEF5
:101194000F74742EF8767078DAE6FEC4540FFDCC22
:1011A400EFCC0F74742CF8EDF6EEC454F0FE78DB3B
:1011B400E6FD131313541F12186454E0FE78DCE6A2
:1011C400FD1313543F1218643354C0FE78DDE6FD5A
:1011D400C31312186433335480FECDEFCD0F7474EF
:1011E4002DF8EEF68F1A7F38121C17121D97EF2078
:0211F400E0F920
:0111F60022D6
:10190800C219121874751A0A787476CD0876800888
:1019180076E00876F80876700876050876D50876B1
:101928009B0876FFE408F67F38121C17121D97EF04
:0319380020E0F9B3
:01193B002289
:101BE200EF24F9600B14600C2402700EC2198007F6
:0B1BF200D21980031218741211642233
:1014AD00C3EF648094E1400ED3EF648094FA50064C
:1014BD00EF24ACFF803CC3EF648094C1400ED3EFAA
:1014CD00648094DA5006EF24CCFF8026C3EF64804D
:1014DD0094B0400ED3EF648094B9500674D02FFFB2
:1014ED008010BF2D047F0A8009BF5F047F0B80022F
:0314FD007F0C223F
:101A7300CEEDCECDEFCDCFEECF1214ADEF3395E05B
:101A8300FE74D22FF58274193EF583E493FF74DA62
:071A93002DF8EFF6021164CB
:061731008B3B8A3C893D60
:10173700E4FE9019DE121885BE04F7E4FEAB3BAA5F
:101747003CA93D8E8275830012078FFF6019121422
:10175700ADEFFD3395E0FC74D22DF58274193CF59D
:0A17670083121885BE04D602116437
:041283008F828E8345
:101287001218907B197AFC79FF78FFD312091B405B
:101297000390FC19AF82AE83121890E47B0F7A2774
:1012A700F9F8C312091B500390270FE4F52F74D5E3
:1012B700252FF8E4F6052FE52FB405F2AE83AF82AC
:1012C700121890121897120D9C78D8E6701A752F7D
:1012D7000374D4252FF8E6FF74D5252FF8EFF6D53C
:1012E7002FEF78D5762080E1121897121731300842
:1012F7000F7BFF7A1979CE121CE4121897121CE49F
:0113070022C3
:101CD100C212C214C211E4FDFF121B6FE4FD7F01A9
:031CE100021B6F74
:101B6F00EF146011047016BD0104C2A78002D2A742
:0E1B7F00A2A7921322BD0103C2A622D2A62263
:101A9A00EF24FE600D14601124027019D212756FC2
:101AAA000122C212A21392A722D2147570027D01DA
:061ABA007F01121B6F22E8
:101A2200301212D56F0F30A707C2A7756F0F80054E
:101A3200D2A7756F23E570D39400400CD57009C20C
:091A420014E4FD7F01121B6F2268
:101C810046554C4C005A4C4F470020332D320054DE
:041C9100726967000D
:101B8D00E6FE08E6FFE4FCFD2278CB12095678C389
:0D1B9D0002096FC3E55D94B8E55C940B226E
:03001300021B2E9F
:101B2E00C0E0C0D075D010200E0CAF8DEFAD8BF590
:101B3E0059EDF55AD20E758D00758B00D0D0D0E0D0
:011B4E003264
:02189E008F3A7F
:1018A000E4F53BF53CC3E53C953AE53B9400502319
:1018B000900000AF82AE83E4FCFD7B207A4EF9F805
:1018C000D312091B4003A380EA053CE53C70D60512
:0318D0003B80D288
:0118D30022F2
:0E1D36007BFF7A1C79811217317F0A02189EFA
:0F1D1900D20C301506121D36C20C221216F02203
:05000E00C20C02182ADB
:101C2E0078CF12097B00000000121B9678CB1209A8
:061C3E007B000000002203
:10003600121D08121D74121CD17F0412189E2097DF
:100046000B7D017F01121308D2AF80FE209612D2DB
:10005600AF121970C2177F701219F91211F7120533
:100066001C121970120512D2AFC2177F701219F93D
:100076007F0112189E1211F71219087A1C7986123E
:1000860005077A1C798B12050712001AE4F573121C
:1000960017EF7F0112189EE478D3F608F6120021B6
:1000A600A2969209A297920AE4F52478C712097BD0
:1000B60000000000E4F52578CF12097BFFFFD8F198
:1000C60078C312097B00000000E4F54E78CB1209D4
:1000D6007B00000000C20DC20CE4F526F527C2081D
:1000E600F55CF55DF559F55AC20EF55BC20FF5588C
:1000F600F557F556F555F561F560F55FF55EF520B2
:100106007899E66004D2808002C28078AAE624FE4E
:10011600600B14600C2402700AD2018006D206809D
:1001260002D20078ABE624FE6007047006D2028095
:1001360002D20778ACE624FE600B14600C24027031
:100146000AD2038006D2048002D205300117C2010A
:1001560078A2121B8D7B64FAF9F81207F08F588E7D
:10016600578D568C55E573C3940240F9E4F573A296
:1001760008B392A6209605209702D2103096353005
:10018600973230102FC21078C3120956EC4D4E4FDD
:1001960078CF700C12097B00000000121B968010AD
:1001A60012097B0000000078C312097B00000000E2
:1001B600D20AD209A209309601B3502DA29692090D
:1001C60030961F20101C121BA05017C201E54E606E
:1001D60007E4F54E7F068005754E017F07121BE288
:1001E600805BE4F55CF55D8054209651740A255DCC
:1001F600F55DE4355CF55C121BA04041E55D9410AD
:10020600E55C94275037755C27755D10300807C28A
:10021600081205128027D2087D01E4FF1213087F19
:100226008912001E7F0112189E7F8212001E7F0116
:1002360012189E7F8412001E7F3112001EA20A3001
:100246009701B35017A297920A30971020100DB25B
:100256000C300C05121D19800312000E1209BAAFDC
:1002660058AE57AD56AC55EC4D4E4F602674FF2F29
:10027600F558EE34FFF557ED34FFF556EC34FFF53F
:1002860055AF58AE57AD56FC4D4E4F7006200C0379
:10029600121D19AF61AE60AD5FAC5EEC4D4E4F60A6
:1002A6002374FF2FF561EE34FFF560ED34FFF55F43
:1002B600EC34FFF55EAF61AE60AD5FFC4D4E4F7046
:1002C6000312000E200E03020372C2AFC20ED2AF9B
:1002D600E4855A2B85592AF529F528AF2BAE2AAD88
:1002E60029AC287B107A27F9F81207F08F2B8E2A73
:1002F6008D298C28E4FB7A90F9F81215E58F2B8E60
:100306002A8D298C2878A0E66009C374B89FFF74EB
:100316000B9EFEE55B14601624FE602024037049E4
:10032600C3EF94B0EE9404500E755B018009D3EFD1
:100336009414EE94054035755B038030C3EF94B09A
:10034600EE94045027755B01300006200C03121D45
:1003560019300305C203121C2E300C02D20F7BFF8C
:100366007A1C79901217318003E4F55B0525E525A3
:10037600C394015003020501E4F525FB7A0079DEFA
:10038600121A4B78DFEEF608EFF678DEE6640260C6
:100396000302050178C7120962E8C0E0E9C0E0EA95
:1003A600C0E0EBC0E078DFE6FE08E6FF7898E6FD01
:1003B600121552D0E0FBD0E0FAD0E0F9D0E0F8EB2D
:1003C6002FFFEA3EFEE93DFDE83CFC78C712096FC7
:1003D6000524E524C39405500302050178C71209D4
:1003E60056E47B05FAF9F81215E578C712096F7815
:1003F600C712095678C3120962C3EF9BFFEE9AFE35
:10040600ED99FDEC98FC78C712096F78CF12095662
:1004160078C7120962D312091B400A78C712095617
:1004260078CF12096FE54E600D78D1E6FF08E678C1
:10043600E1CFF608EFF678C9E6FF08E678DFCFF6F3
:1004460008EFF6E54E600308800278DFE6FE08E670
:10045600FF1212830527E52770020526C3789796B3
:10046600E52618964045E4F526F527300D0F78DF8A
:10047600E608FF12001E78E0E6FF12001E300C2B85
:100486007F03121A9A20151D78A1E6600C300F0919
:100496007F007E82121384C20F78DFE6FE08E6FF35
:1004A6001213848006121D3612000E78C7120956E2
:1004B60078CB12096F78C712097B00000000E4F5BB
:1004C60024300405C204121C2E30061678A6121B10
:1004D6008D78CB120962D312091B4006200C031239
:1004E6001D1930071678A8121B8D78CB120962C326
:1004F60012091B5006300C0312000E121A220201BA
:010506006B89
:100507007BFF1217317F0412189E2278AFE6FDE4B5
:05051700FF1213082291
:101AC000444C0021536967005A4C4F47004D4F4426
:101AD00000332D32004665622030332032303036FC
:061AE0000050524F4700C8
:10166C00AF34AE33AD32AC31EC4D4E4F22EF24FFE4
:10167C00F534EE34FFF533ED34FFF532EC34FFF591
:10168C003122E475342075334EF532F53122E47590
:10169C003401F533F532F53122752E00752F0075B6
:0316AC0030942255
:04001600E4F54E229D
:1009BA00121D44EF7003020BD0121BAAEF12099406
:1009CA000BA9240BB52A0BBB500B015209F2610A81
:1009DA0083630AD66C0ADC720AD9730B05740B7925
:1009EA00760B737800000BD01200167BFF7A1A7907
:1009FA00C012173112168E121D44EF700A12166CAD
:100A0A00600512167980F012166C7003020BD01270
:100A1A001BAA8F2D12159EE4F53412169EE47F064A
:100A2A00FEFDFCAB34AA33A932A831C312093150F6
:100A3A001F121C598F2D12001EE5342401F534E4CF
:100A4A003533F533E43532F532E43531F53180CDDD
:100A5A00121C598F2DE52D64806016E52D64816086
:100A6A001012001E121C598F2D12001E752C0180A7
:100A7A0003E4F52CE52C70D8221216A512169AF565
:100A8A002D12166C602412168E121D44EF700A1273
:100A9A00166C600512167980F012166C6003120B40
:100AAA00D1052DE52DC3941C40D712166C601A7817
:100ABA0094B6AB0708B6CD03020BB27BFF7A1A795C
:100ACA00C31217317F0A02189E020B70B20D22025E
:100ADA0013FC1216A5E4F52DAB2E0530E530AA2F2E
:100AEA007002052F14F9120776FF12001E052DE574
:100AFA002DC3941C40E22243A20822120016752E2E
:100B0A0000752F0075307112169AF52D12166C6049
:100B1A002412168E121D44EF700A12166C6005120A
:100B2A00167980F012166C6003120BD1052DE52D93
:100B3A00C3940240D712166C602CAE71AF72EE33BA
:100B4A0095E0FDFC78CB120962C3EF9BF538EE9A6B
:100B5A00F537ED99F536EC98F535AF38789EE537E7
:100B6A00F608EFF680420216291200160214557A88
:100B7A001A79C8120BE57A1A79CD121CE478ADE617
:100B8A002430FF12001E121D877F7612001E7A1A69
:100B9A0079D1120BE57A1A79D5121CE4021D871253
:100BAA000016E4789EF608F6021AE61200160217F4
:100BBA00711200167BFF7A1A79E11217317D017FD3
:060BCA000112130880FE79
:100BD00022121BAAAB2EAA2FA930852D8275830065
:100BE000EF1207CE227BFF121CE4121D877BFF222F
:0A1D7400E4F5955396BF53A27F22B9
:1017EF005389F0438901538FFE758C70E4F58A534A
:1017FF00B8FD53B7FDD2A9D28C53890F43899053AB
:10180F008FEFF58DF58B4391105392EF53B8F7533C
:0B181F00B7F7D2ABD28ED28AD2AA2239
:03000B00021D7E55
:091D7E000573758C70758A003242
:03001B00021D9033
:071D9000758D00758B003218
:101C95000D0A003031323334353637383941424355
:041CA500444546006C
:101CA900AF4DAB41AA42A943054D22AF40AE3FAD6E
:041CB9003EAC3D22DE
:101308005387BF75985053877FE4F5BABF010543EB
:10131800A240800353A2BFE4F5BDED14601514602C
:101328001A14601F1460242404702575BEF075BF5C
:101338000B802375BEF075BF05801B75BEF075BFA9
:1013480002801375BE7075BF01800B75BEB0800337
:1013580075BE30E4F5BF75BD035391FE439201435A
:1013680091025392FDC21A53B8EF53B7EF43B81026
:0C137800E478C1F618F678C2F6D2AC2278
:0300230002193C83
:10193C00C0E0C0D075D01030981E78C1E6C3940FAB
:10194C00501418E60624B0F8A69978C10618E6C318
:10195C00941040027600C298309904C299C21AD0F1
:04196C00D0D0E032C5
:08000300201AFDD21A8F992288
:101B4F0078C1E6D39400401508E60624B0F8E6FF06
:0F1B5F0078C11608E6C394104005E4F6227F0013
:011B6E002254
:03001E00020003DA
:101BAA007F207E4E78C1E67010D3EF9400EE940049
:0C1BBA004007EF1F70EE1E80EB121B4F67
:011BC60022FC
:101CE400120776FF600C12001E740129F9E43AFA17
:031CF40080EE225D
:0E1D440078C1E6D3940040037F01227F002285
:091D87007BFF7A1C7995021CE433
:0E0D9C008F408E3F8D3E8C3D8B418A428943B5
:100DAA00E4F54DEC4D4E4F7017E94A4B70057F3014
:100DBA0002001E121CA98F827583007430020EBFB6
:100DCA00121CB6EC33502AE5434542454170077F71
:100DDA002D12001E800D121CA98F82758300742D9E
:100DEA001207CE121CB412090D8F408E3F8D3E8C15
:100DFA003D754C017547007546CA75459A75443B61
:100E0A00E4FFFEFDFCAB47AA46A945A844D3120954
:100E1A00315003020EAA121CB4A84412087B8F4B4D
:100E2A008E4A8D498C48EC4D4E4F7004E54C702328
:100E3A00E54B2430FFE54345424541700512001E4B
:100E4A00800EAE4D121CAB8E82758300EF1207CE58
:100E5A00E4F54CAF47AE46AD45AC44AB4BAA4AA904
:100E6A0049A8481207F0C8ECC8C9EDC9CAEECAC3F6
:100E7A00E5409FF540E53F9AF53FE53E99F53EE5A9
:100E8A003D98F53DAF47AE46AD45AC44E47B0AFA22
:100E9A00F9F812087B8F478E468D458C44020E0A5C
:100EAA00E542454345416010AB41AA42A943854DFD
:080EBA0082758300E41207CEEB
:010EC200220D
:100BF0000134C35001DBBF68028BBB800344B7984C
:100C00000407B3B004D5AFC805A9ABE00689A7F8BF
:100C10000775A410086DA02809719C400A81985896
:100C20000B9F94700CCA90880DE98CF90E048CA06F
:100C30000EA88AAC0F4D88B80FF786C410A184D0D7
:100C4000115182DC120580E812BB7EF413747D0022
:100C500014307B0C14F2791815B87724168075308F
:100C6000174B733C1819714818ED6F5419C46D6017
:100C70001AA16B6C1B7E69781C6167841D4A6590A4
:100C80001E37639C1F2561A8201A5FB421125DC026
:100C9000220D5BCC230E59D8241557E4251F55F09F
:100CA000262F53FC27425208285B501429764E20E9
:100CB0002A9B4C2C2BC04A382CEE48442E1E465002
:100CC0002F55445C308F426831D1407433173E80D9
:100CD00034633C8C35B13A98370938A4386636B05D
:100CE00039C734BC3B2D32C83C9D30D43E0F2EE07A
:100CF0003F882CEC41062AF8428D2904441827101D
:100D000045AB251C4741232848E121344A861F4032
:100D10004C311D4C4DE21B584F9C1964515D1770AE
:100D20005323157C54EF138856C4119458A20FA076
:100D30005A830DAC5C6D0BB85E6009C4605807D077
:100D4000625A05DC646203E8667301F4688A000095
:100D50006AA1FE0C6CB8FC186ECFFA2470E6F8306D
:100D60000000000000000000000000000000000083
:100D70000000000000000000000000000000000073
:100D80000000000000000000000000000000000063
:0C0D900000000000000000000000000057
:1017B00075F004E533A424F0F582E5F0340BF583ED
:1017C000E49322FE740193FF75F004E533A422F53F
:1017D00083C37401939FFFE4939EFEE4228F348EB3
:0F17E000338D328C31228F308E2F8D2E8C2D2217
:101CBD00C3EF9DEE9C400AD3EF9BEE9A50037F013C
:041CCD00227F002250
:040EC3008E318F32AB
:100EC700E4F5331217B0FC740193FD1217C824F42C
:100ED700F582E5F0340BF583E493FA740193FBAFE5
:100EE70032AE31121CBDEF7003020FB31217B012EE
:100EF70017C324F4F582E5F0340B1217CF8F378E22
:100F070036F535F5341217C824F6F582E5F0340BBB
:100F1700F583E4931217C324F2F582E5F0340B123C
:100F270017CF8F3B8E3AF539F538AD39AC38120902
:100F37000D8F3B8E3A8D398C38AE31AF32E4FCFDE4
:100F4700EEC0E0EFC0E01217B0FE740193FBCAEEEB
:100F5700CAD0E0FFD0E0FEC3EF9BFFEE9AFEED9410
:100F670000FDEC9400FCAB3BAA3AA939A83812075C
:100F7700F0AB37AA36A935A8341215E5C8ECC8C9AD
:100F8700EDC9CAEECACBEFCB1217C824F2F582E53A
:100F9700F0340BF583E493FE740193FFE4FCFDEB5F
:100FA7002FFFEA3EFEED39FDEC38FC220533E53331
:0D0FB700C3946A5003020ECAE4FFFEFDFC65
:010FC400220A
:0100210022BC
:101500001217DDAB34AA33A932A831E8C0E0789CC9
:10151000E6FE08E6FFE4FCFDD0E0F81207F0121743
:10152000DD780E1209421217DD789EE6FE08E6FF0E
:10153000EE3395E0FDFCE5342FF534E5333EF5332D
:10154000E5323DF532E5313CF531AF34AE33AD3205
:02155000FC227B
:021552008D2CDE
:10155400120EC31217E61215001217E6E52C1460DA
:101564001C14702DE47FE87E03FDFCAB30AA2FA988
:101574002EA82D1207F0E47BE87A0B800CAF30AE76
:101584002FAD2EAC2DE47B03FAF9F81215E51217F2
:09159400E6AF30AE2FAD2EAC2DF8
:01159D00222B
:10077600BB010689828A83E0225002E722BBFE0281
:09078600E32289828A83E49322B4
:10078F00BB010CE58229F582E5833AF583E022501F
:10079F0006E92582F8E622BBFE06E92582F8E22269
:0D07AF00E58229F582E5833AF583E4932283
:1007BC00BB010689828A83F0225002F722BBFE011C
:0207CC00F32216
:1007CE00F8BB010DE58229F582E5833AF583E8F061
:1007DE00225006E92582C8F622BBFE05E92582C80D
:0207EE00F222F5
:1007F000E88FF0A4CC8BF0A42CFCE98EF0A42CFCA8
:100800008AF0EDA42CFCEA8EF0A4CDA8F08BF0A425
:100810002DCC3825F0FDE98FF0A42CCD35F0FCEB84
:100820008EF0A4FEA9F0EB8FF0A4CFC5F02ECD3949
:0F083000FEE43CFCEAA42DCE35F0FDE43CFC22B6
:10083F0075F008758200EF2FFFEE33FECD33CDCC70
:10084F0033CCC58233C5829BED9AEC99E5829840F3
:10085F000CF582EE9BFEED9AFDEC99FC0FD5F0D6D0
:10086F00E4CEFBE4CDFAE4CCF9A88222B800C1B9FA
:10087F000059BA002DEC8BF084CFCECDFCE5F0CB38
:10088F00F97818EF2FFFEE33FEED33FDEC33FCEB71
:10089F0033FB10D703994004EB99FB0FD8E5E4F92C
:1008AF00FA227818EF2FFFEE33FEED33FDEC33FC19
:1008BF00C933C910D7059BE99A4007EC9BFCE99A0D
:1008CF00F90FD8E0E4C9FAE4CCFB2275F010EF2F52
:1008DF00FFEE33FEED33FDCC33CCC833C810D70752
:1008EF009BEC9AE899400AED9BFDEC9AFCE899F88D
:0E08FF000FD5F0DAE4CDFBE4CCFAE4C8F92220
:1015E500C2D5E830E70FB2D5E4C39BFBE49AFAE431
:1015F50099F9E498F8EC30E717B2D512161B1208E2
:101605007BE4C39BFBE49AFAE499F9E498F8800338
:1016150012087B30D50DE4C39FFFE49EFEE49DFDDB
:04162500E49CFC2223
:0E090D00C3E49FFFE49EFEE49DFDE49CFC22FB
:10091B00EB9FF5F0EA9E42F0E99D42F0EC6480C853
:06092B0064809845F022F3
:10093100EB9FF5F0EA9E42F0E99D42F0E89C45F01C
:010941002293
:10094200E86010ECA2E713FCED13FDEE13FEEF13CB
:04095200FFD8F022B8
:0C095600E6FC08E6FD08E6FE08E6FF22CD
:0D096200E6FB08E6F908E6FA08E6CBF82205
:0C096F00ECF608EDF608EEF608EFF622B4
:10097B00D083D082E493F608740193F60874029343
:09098B00F608740393F67404737A
:10099400D083D082F8E4937012740193700DA3A3F2
:1009A40093F8740193F5828883E473740293686006
:0609B400EFA3A3A380DF06
:00000001FF
